******************************************************************************
          TMS320C6x COFF Linker PC v6.0.16                     
******************************************************************************
>> Linked Tue Mar 11 10:15:04 2008

OUTPUT FILE NAME:   <../obj/debug/Emac_2DSP.out>
ENTRY POINT SYMBOL: "_c_int00"  address: 0083d980


MEMORY CONFIGURATION

         name            origin    length      used     unused   attr    fill
----------------------  --------  ---------  --------  --------  ----  --------
  L2Vector              00800000   00000200  00000200  00000000  RWIX
  L2First               00800200   0007fe00  00040e38  0003efc8  RWIX
  L2Test                00880000   00080000  00000000  00080000  RWIX
  L1P                   00e00000   00008000  00000000  00008000  RWIX
  L1D                   00f00000   00008000  00000000  00008000  RWIX
  DDR2                  e0000000   00800000  00000000  00800000  RWIX


SECTION ALLOCATION MAP

 output                                  attributes/
section   page    origin      length       input sections
--------  ----  ----------  ----------   ----------------
.csl_vect 
*          0    00800000    00000200     
                  00800000    00000200     csl_c64xplus_intc.lib : _csl_intcIsrDispatch.o (.csl_vect)

.data      0    00800200    00000000     UNINITIALIZED

KeyFunc    0    00800200    00000000     UNINITIALIZED

EMAC_DATA 
*          0    00800200    00031600     UNINITIALIZED
                  00800200    00031600     Emac_2DSP.obj (EMAC_DATA)

.text      0    00831800    0000c700     
                  00831800    00001440     Emac_2DSP.obj (.text)
                  00832c40    000009c0     csl_c6482_bc.lib : csl_emac.o (.text:_EMAC_open)
                  00833600    00000940                      : csl_mdio.o (.text:_MDIO_timerTick)
                  00833f40    00000420     rts64plus.lib : _printfi.obj (.text:__setfield)
                  00834360    00000400     csl_c6482_bc.lib : csl_mdio.o (.text:_MDIO_initContinue)
                  00834760    000003c0     csl_c64xplus_intc.lib : csl_intcHwControl.o (.text:csl_section:intc:_CSL_intcHwControl)
                  00834b20    000003a0     csl_c6482_bc.lib : csl_emac.o (.text:_EMAC_close)
                  00834ec0    00000360     rts64plus.lib : _printfi.obj (.text:__getarg_diouxp)
                  00835220    00000360                   : _printfi.obj (.text:__printfi)
                  00835580    00000340     csl_c6482_bc.lib : csl_mdio.o (.text:_MDIO_initPHY)
                  008358c0    00000300     rts64plus.lib : _printfi.obj (.text:_ecvt)
                  00835bc0    00000300                   : _printfi.obj (.text:_fcvt)
                  00835ec0    00000300                   : fputs.obj (.text:_fputs)
                  008361c0    00000300     csl_c64xplus_intc.lib : csl_intcInit.o (.text:csl_section:intc:_CSL_intcInit)
                  008364c0    000002e0     rts64plus.lib : _printfi.obj (.text:__fcpy)
                  008367a0    000002e0                   : _printfi.obj (.text:__pproc_fwp)
                  00836a80    000002a0                   : _printfi.obj (.text:__pconv_e)
                  00836d20    00000280                   : memory.obj (.text:_free)
                  00836fa0    00000280     csl_c6482_bc.lib : csl_devHwControl.o (.text:csl_section:dev:_CSL_devHwControl)
                  00837220    00000260                      : csl_emac.o (.text:_EMAC_timerTick)
                  00837480    00000260                      : csl_devGetHwStatus.o (.text:csl_section:dev:_CSL_devGetHwStatus)
                  008376e0    00000260                      : csl_tmrHwControl.o (.text:csl_section:tmr:_CSL_tmrHwControl)
                  00837940    00000260                      : csl_tmrHwSetup.o (.text:csl_section:tmr:_CSL_tmrHwSetup)
                  00837ba0    00000240                      : csl_emac.o (.text:_EMAC_serviceCheck)
                  00837de0    00000240     rts64plus.lib : frcdivd.obj (.text:__frcdivd)
                  00838020    00000240     csl_c64xplus_intc.lib : csl_intcOpen.o (.text:csl_section:intc:_CSL_intcOpen)
                  00838260    00000220     Emac_Int_setup.obj (.text)
                  00838480    00000220     rts64plus.lib : imath64.obj (.text:__divull)
                  008386a0    00000220                   : _printfi.obj (.text:__pproc_diouxp)
                  008388c0    00000220                   : _printfi.obj (.text:__pproc_str)
                  00838ae0    00000220     csl_c6482_bc.lib : csl_emac.o (.text:_emacDequeueRx)
                  00838d00    00000220     csl_c64xplus_intc.lib : _csl_intcCombEventDispatcher.o (.text:csl_section:intc:__CSL_intcEvent0Dispatcher)
                  00838f20    00000220                           : _csl_intcCombEventDispatcher.o (.text:csl_section:intc:__CSL_intcEvent1Dispatcher)
                  00839140    00000220                           : _csl_intcCombEventDispatcher.o (.text:csl_section:intc:__CSL_intcEvent2Dispatcher)
                  00839360    00000220                           : _csl_intcCombEventDispatcher.o (.text:csl_section:intc:__CSL_intcEvent3Dispatcher)
                  00839580    00000200     rts64plus.lib : frcaddd.obj (.text:__frcaddd)
                  00839780    000001e0                   : _printfi.obj (.text:__mcpy)
                  00839960    000001e0     csl_c64xplus_intc.lib : _csl_intcDispatcher.o (.text:csl_section:intc:__CSL_intcDispatcher)
                  00839b40    000001c0     csl_c6482_bc.lib : csl_emac.o (.text:_EMAC_sendPacket)
                  00839d00    000001c0     rts64plus.lib : divd.obj (.text:__divd)
                  00839ec0    000001a0                   : trgdrv.obj (.text:_HOSTrename)
                  0083a060    000001a0                   : imath40.obj (.text:__divul)
                  0083a200    000001a0                   : mpyd.obj (.text:__mpyd)
                  0083a3a0    000001a0     csl_c6482_bc.lib : csl_emac.o (.text:_emacEnqueueTx)
                  0083a540    000001a0     rts64plus.lib : setvbuf.obj (.text:_setvbuf)
                  0083a6e0    00000180     csl_c6482_bc.lib : csl_emac.o (.text:_emacDequeueTx)
                  0083a860    00000180     rts64plus.lib : memory.obj (.text:_malloc)
                  0083a9e0    00000160                   : addd.obj (.text:__addd)
                  0083ab40    00000160                   : _printfi.obj (.text:__pconv_g)
                  0083aca0    00000160                   : _printfi.obj (.text:__pproc_fge)
                  0083ae00    00000160     csl_c6482_bc.lib : csl_emac.o (.text:_emacEnqueueRx)
                  0083af60    00000140     csl_c64xplus_intc.lib : _csl_intcIntrEnDisRes.o (.text:csl_section:intc)
                  0083b0a0    00000140     csl_c6482_bc.lib : csl_tmrGetHwSetup.o (.text:csl_section:tmr:_CSL_tmrGetHwSetup)
                  0083b1e0    00000120                      : csl_emac.o (.text:_EMAC_getStatus)
                  0083b300    00000120                      : csl_emac.o (.text:_EMAC_setReceiveFilter)
                  0083b420    00000120     rts64plus.lib : _printfi.obj (.text:__pproc_fflags)
                  0083b540    00000120                   : fclose.obj (.text:_fclose)
                  0083b660    00000120                   : fputc.obj (.text:_fputc)
                  0083b780    00000100                   : trgdrv.obj (.text:_HOSTopen)
                  0083b880    00000100                   : frcmpyd.obj (.text:__frcmpyd)
                  0083b980    00000100                   : _printfi.obj (.text:__ltostr)
                  0083ba80    00000100                   : atoi.obj (.text:_atoi)
                  0083bb80    00000100                   : exit.obj (.text:_exit)
                  0083bc80    00000100                   : lowlev.obj (.text:_getdevice)
                  0083bd80    000000e0                   : trgdrv.obj (.text:_HOSTlseek)
                  0083be60    000000e0                   : autoinit.obj (.text:__auto_init)
                  0083bf40    000000e0                   : _printfi.obj (.text:__div)
                  0083c020    000000e0                   : _io_perm.obj (.text:__wrt_ok)
                  0083c100    000000e0                   : lowlev.obj (.text:_close)
                  0083c1e0    000000e0     csl_c6482_bc.lib : csl_emac.o (.text:_emacUpdateStats)
                  0083c2c0    000000e0     rts64plus.lib : fseek.obj (.text:_fseek)
                  0083c3a0    000000e0                   : memset.obj (.text:_memset)
                  0083c480    000000c0                   : trgdrv.obj (.text:_HOSTread)
                  0083c540    000000c0                   : trgdrv.obj (.text:_HOSTunlink)
                  0083c600    000000c0                   : trgdrv.obj (.text:_HOSTwrite)
                  0083c6c0    000000c0     csl_c6482_bc.lib : csl_mdio.o (.text:_MDIO_close)
                  0083c780    000000c0     rts64plus.lib : fopen.obj (.text:__cleanup)
                  0083c840    000000c0                   : divu.obj (.text:__divu)
                  0083c900    000000c0                   : _printfi.obj (.text:__pconv_f)
                  0083c9c0    000000c0                   : lowlev.obj (.text:_lseek)
                  0083ca80    000000c0                   : ltoa.obj (.text:_ltoa)
                  0083cb40    000000c0                   : lowlev.obj (.text:_write)
                  0083cc00    000000c0     csl_c64xplus_intc.lib : csl_intcClose.o (.text:csl_section:intc:_CSL_intcClose)
                  0083ccc0    000000c0     csl_c6482_bc.lib : csl_tmrOpen.o (.text:csl_section:tmr:_CSL_tmrOpen)
                  0083cd80    000000a0     rts64plus.lib : trgdrv.obj (.text:_HOSTclose)
                  0083ce20    000000a0                   : imath40.obj (.text:__divli)
                  0083cec0    000000a0                   : fflush.obj (.text:__doflush)
                  0083cf60    000000a0                   : _printfi.obj (.text:__ecpy)
                  0083d000    000000a0                   : fixdli.obj (.text:__fixdli)
                  0083d0a0    000000a0                   : fltlid.obj (.text:__fltlid)
                  0083d140    000000a0                   : lowlev.obj (.text:_finddevice)
                  0083d1e0    000000a0                   : memcpy64.obj (.text:_memcpy)
                  0083d280    000000a0                   : memory.obj (.text:_minsert)
                  0083d320    000000a0                   : memory.obj (.text:_mremove)
                  0083d3c0    000000a0                   : renormd.obj (.text:_renormd)
                  0083d460    000000a0                   : trgmsg.obj (.text:_writemsg)
                  0083d500    000000a0     csl_c6482_bc.lib : csl_devOpen.o (.text:csl_section:dev:_CSL_devOpen)
                  0083d5a0    00000080                      : csl_mdio.o (.text:_MDIO_open)
                  0083d620    00000080     rts64plus.lib : cmpd.obj (.text:__cmpd)
                  0083d6a0    00000080                   : fixdi.obj (.text:__fixdi)
                  0083d720    00000080                   : llshift.obj (.text:__llshl)
                  0083d7a0    00000080                   : printf.obj (.text:_printf)
                  0083d820    00000080                   : trgmsg.obj (.text:_readmsg)
                  0083d8a0    00000080                   : lowlev.obj (.text:_unlink)
                  0083d920    00000060                   : imath64.obj (.text:__subcull)
                  0083d980    00000060                   : boot.obj (.text:_c_int00)
                  0083d9e0    00000060                   : memccpy.obj (.text:_memccpy)
                  0083da40    00000060     csl_c6482_bc.lib : csl_timerGetBaseAddress.o (.text:csl_section:tmr:_CSL_tmrGetBaseAddress)
                  0083daa0    00000040     rts64plus.lib : args_main.obj (.text:__args_main)
                  0083dae0    00000040                   : llshift.obj (.text:__llshru)
                  0083db20    00000040                   : negd.obj (.text:__negd)
                  0083db60    00000040                   : imath40.obj (.text:__remli)
                  0083dba0    00000040                   : strasg.obj (.text:__strasgi_64plus)
                  0083dbe0    00000040                   : subd.obj (.text:__subd)
                  0083dc20    00000040     csl_c6482_bc.lib : csl_emac.o (.text:_pqPush)
                  0083dc60    00000040     rts64plus.lib : fputs.obj (.text:_puts)
                  0083dca0    00000040     csl_c6482_bc.lib : csl_cacheL1.o (.text:csl_section:cache:_CACHE_setL1dSize)
                  0083dce0    00000040                      : csl_cacheL1.o (.text:csl_section:cache:_CACHE_setL1pSize)
                  0083dd20    00000040                      : csl_cacheL2.o (.text:csl_section:cache:_CACHE_setL2Size)
                  0083dd60    00000040                      : csl_devGetBaseAddress.o (.text:csl_section:dev:_CSL_devGetBaseAddress)
                  0083dda0    00000020                      : csl_mdio.o (.text:_MDIO_getStatus)
                  0083ddc0    00000020     rts64plus.lib : negll.obj (.text:__negll)
                  0083dde0    00000020                   : _lock.obj (.text:__nop)
                  0083de00    00000020                   : printf.obj (.text:__outc)
                  0083de20    00000020                   : printf.obj (.text:__outs)
                  0083de40    00000020                   : exit.obj (.text:_abort)
                  0083de60    00000020                   : remove.obj (.text:_remove)
                  0083de80    00000020     csl_c6482_bc.lib : csl_devInit.o (.text:csl_section:dev:_CSL_devInit)
                  0083dea0    00000020     csl_c64xplus_intc.lib : _csl_intcNmiDummy.o (.text:csl_section:intc)
                  0083dec0    00000020                           : csl_intcHookIsr.o (.text:csl_section:intc:_CSL_intcHookIsr)
                  0083dee0    00000020     csl_c6482_bc.lib : csl_tsc.o (.text:cslsys_section:tsc)

.stack     0    0083df00    00001000     UNINITIALIZED
                  0083df00    00000008     rts64plus.lib : boot.obj (.stack)

.sysmem    0    0083ef00    00001000     UNINITIALIZED
                  0083ef00    00000008     rts64plus.lib : memory.obj (.sysmem)

.far       0    0083ff00    0000085c     UNINITIALIZED
                  0083ff00    000002e0     csl_c6482_bc.lib : csl_emac.o (.far)
                  008401e0    00000194     rts64plus.lib : defs.obj (.far)
                  00840374    00000004                   : fopen.obj (.far)
                  00840378    00000118     Emac_Int_setup.obj (.far)
                  00840490    000000d0     rts64plus.lib : trgdrv.obj (.far)
                  00840560    000000cc                   : lowlev.obj (.far)
                  00840630    00000090                   : exit.obj (.far)
                  008406c0    00000058     Emac_2DSP.obj (.far)
                  00840718    00000034     csl_c6482_bc.lib : csl_mdio.o (.far)
                  0084074c    00000008     rts64plus.lib : _lock.obj (.far)
                  00840754    00000008                   : memory.obj (.far)

.const     0    00840760    000003dc     
                  00840760    000002b1     Emac_2DSP.obj (.const)
                  00840a11    00000002     rts64plus.lib : fputs.obj (.const)
                  00840a13    00000005     --HOLE-- [fill = 0]
                  00840a18    00000101                   : ctype.obj (.const:__ctypes_)
                  00840b19    00000023                   : _printfi.obj (.const)

.cinit     0    00840b40    00000274     
                  00840b40    000000a0     Emac_2DSP.obj (.cinit)
                  00840be0    0000005c     rts64plus.lib : lowlev.obj (.cinit)
                  00840c3c    00000004     --HOLE-- [fill = 0]
                  00840c40    0000005c                   : defs.obj (.cinit)
                  00840c9c    00000004     --HOLE-- [fill = 0]
                  00840ca0    0000002c     csl_c6482_bc.lib : csl_mdio.o (.cinit)
                  00840ccc    00000004     --HOLE-- [fill = 0]
                  00840cd0    0000002c     rts64plus.lib : exit.obj (.cinit)
                  00840cfc    00000004     --HOLE-- [fill = 0]
                  00840d00    0000002c                   : memory.obj (.cinit)
                  00840d2c    00000004     --HOLE-- [fill = 0]
                  00840d30    0000001c     csl_c6482_bc.lib : _csl_cache.o (.cinit)
                  00840d4c    00000004     --HOLE-- [fill = 0]
                  00840d50    0000001c     csl_c64xplus_intc.lib : _csl_intcResource.o (.cinit)
                  00840d6c    00000004     --HOLE-- [fill = 0]
                  00840d70    0000001c     rts64plus.lib : _lock.obj (.cinit)
                  00840d8c    00000004     --HOLE-- [fill = 0]
                  00840d90    0000000c     csl_c6482_bc.lib : csl_emac.o (.cinit)
                  00840d9c    00000004     --HOLE-- [fill = 0]
                  00840da0    0000000c     rts64plus.lib : fopen.obj (.cinit)
                  00840dac    00000008     --HOLE-- [fill = 0]

.cio       0    00840db8    00000120     UNINITIALIZED
                  00840db8    00000120     rts64plus.lib : trgmsg.obj (.cio)

.switch    0    00840ed8    000000e0     
                  00840ed8    0000003c     csl_c6482_bc.lib : csl_devGetHwStatus.o (.switch)
                  00840f14    00000038                      : csl_tmrHwControl.o (.switch)
                  00840f4c    0000001c                      : csl_devHwControl.o (.switch)
                  00840f68    0000001c     csl_c64xplus_intc.lib : csl_intcHwControl.o (.switch)
                  00840f84    00000014     csl_c6482_bc.lib : csl_mdio.o (.switch)
                  00840f98    00000010     csl_c64xplus_intc.lib : csl_intcOpen.o (.switch)
                  00840fa8    00000010     rts64plus.lib : frcdivd.obj (.switch)

.bss       0    00840fb8    0000008c     UNINITIALIZED
                  00840fb8    00000054     csl_c64xplus_intc.lib : _csl_intcResource.o (.bss:csl_section:intc)
                  0084100c    00000024     Emac_2DSP.obj (.bss)
                  00841030    0000000c     Emac_Int_setup.obj (.bss)
                  0084103c    00000008     csl_c6482_bc.lib : _csl_cache.o (.bss:csl_section:cache)


GLOBAL SYMBOLS: SORTED ALPHABETICALLY BY Name 

address    name
--------   ----
00840fb8   $bss
00840fb8   .bss
00800200   .data
00831800   .text
0083de40   C$$EXIT
0083d4e4   C$$IO$$
0083dca0   _CACHE_setL1dSize
0083dce0   _CACHE_setL1pSize
0083dd20   _CACHE_setL2Size
0083dd60   _CSL_devGetBaseAddress
00837480   _CSL_devGetHwStatus
00836fa0   _CSL_devHwControl
0083de80   _CSL_devInit
0083d500   _CSL_devOpen
0083cc00   _CSL_intcClose
0083b018   _CSL_intcGlobalDisable
0083aff8   _CSL_intcGlobalEnable
0083b08c   _CSL_intcGlobalExcepClear
0083b064   _CSL_intcGlobalExcepEnable
0083b078   _CSL_intcGlobalExtExcepEnable
0083b050   _CSL_intcGlobalNmiEnable
0083b038   _CSL_intcGlobalRestore
0083dec0   _CSL_intcHookIsr
00834760   _CSL_intcHwControl
008361c0   _CSL_intcInit
0083afb0   _CSL_intcInterruptClear
0083af90   _CSL_intcInterruptDisable
0083af70   _CSL_intcInterruptEnable
0083afcc   _CSL_intcInterruptRestore
0083afc0   _CSL_intcInterruptSet
00838020   _CSL_intcOpen
0083afe4   _CSL_intcQueryInterruptStatus
0083da40   _CSL_tmrGetBaseAddress
0083b0a0   _CSL_tmrGetHwSetup
008376e0   _CSL_tmrHwControl
00837940   _CSL_tmrHwSetup
0083ccc0   _CSL_tmrOpen
0083dee0   _CSL_tscEnable
0083dee8   _CSL_tscRead
008406c8   _DestMAC
00834b20   _EMAC_close
0083b1e0   _EMAC_getStatus
00832c40   _EMAC_open
00839b40   _EMAC_sendPacket
00837ba0   _EMAC_serviceCheck
0083b300   _EMAC_setReceiveFilter
00837220   _EMAC_timerTick
00841018   _EmacControlRegs
00832688   _EmacHwInt
00838448   _EmacInterruptEnd
00838340   _EmacInterruptsInitialization
00841014   _EmacRegs
00838260   _EmacTimerInitialization
008328f0   _EmacTimerTick
008406d0   _FreeQueue
0083cd80   _HOSTclose
0083bd80   _HOSTlseek
0083b780   _HOSTopen
0083c480   _HOSTread
00839ec0   _HOSTrename
0083c540   _HOSTunlink
0083c600   _HOSTwrite
00841024   _LinkStatus
008406c0   _LocalMAC
00841028   _LocalTicks
0083c6c0   _MDIO_close
0083dda0   _MDIO_getStatus
00835580   _MDIO_initPHY
0083d5a0   _MDIO_open
00833600   _MDIO_timerTick
008406dc   _RxQueue
00840db8   __CIOBUF_
00841040   __CSL_cacheEmifState
0084103c   __CSL_cachebusyState
00840fb8   __CSL_intcAllocMask
00840fbc   __CSL_intcCpuIntrTable
00839960   __CSL_intcDispatcher
00838d00   __CSL_intcEvent0Dispatcher
00838f20   __CSL_intcEvent1Dispatcher
00839140   __CSL_intcEvent2Dispatcher
00839360   __CSL_intcEvent3Dispatcher
00841008   __CSL_intcEventHandlerRecord
00841000   __CSL_intcEventOffsetMap
0083af60   __CSL_intcIvpSet
0083dea0   __CSL_intcNmiDummy
00841004   __CSL_intcNumEvents
00800000   __CSL_intcVectorTable
00001000   __STACK_SIZE
00001000   __SYSMEM_SIZE
ffffffff   ___binit__
00840fb8   ___bss__
ffffffff   ___c_args__
00840b40   ___cinit__
00800200   ___data__
00800200   ___edata__
00841044   ___end__
0083df00   ___etext__
ffffffff   ___pinit__
00831800   ___text__
0083a9e0   __addd
0083daa0   __args_main
0083be60   __auto_init
0083c780   __cleanup
008406b8   __cleanup_ptr
0083d620   __cmpd
00840a18   __ctypes_
00839d00   __divd
0083ce20   __divli
0083c840   __divu
0083a060   __divul
00838480   __divull
0083cec0   __doflush
008406bc   __dtors_ptr
0083d6a0   __fixdi
0083d000   __fixdli
0083d0a0   __fltlid
00839580   __frcaddd
00837de0   __frcdivd
0083b880   __frcmpyd
00840370   __ft_end
008401e0   __ftable
0083d720   __llshl
0083dae0   __llshru
0084074c   __lock
0083a200   __mpyd
0083db20   __negd
0083ddc0   __negll
0083dde0   __nop
00835220   __printfi
0083db60   __remli
0083df00   __stack
0083dba0   __strasgi_64plus
0083d920   __subcull
0083dbe0   __subd
0083ef00   __sys_memory
008402d0   __tmpnams
00840750   __unlock
0083c020   __wrt_ok
0083de40   _abort
0083ba80   _atoi
0083d980   _c_int00
0083c100   _close
00832658   _closeEMAC
0084101c   _devRegs
00832594   _emacRxPackets
00832314   _emacTxPackets
00831ac8   _emac_Init
0083bb80   _exit
0083b540   _fclose
0083b660   _fputc
00835ec0   _fputs
00836d20   _free
0083c2c0   _fseek
0083192c   _gblUserInit
00841020   _hEMAC
0083c9c0   _lseek
0083ca80   _ltoa
008319c0   _main
0083a860   _malloc
0083d9e0   _memccpy
0083d1e0   _memcpy
0083c3a0   _memset
00801800   _packet_buffer
00800200   _packet_header
0083d7a0   _printf
0083b660   _putc
0083dc60   _puts
0083d820   _readmsg
0083de60   _remove
0083d3c0   _renormd
0083a540   _setvbuf
0084102c   _uiMacMode
00841010   _uiTotalPacketsReceived
0084100c   _uiTotalPacketsToTransfer
0083d8a0   _unlink
0083cb40   _write
0083d460   _writemsg
ffffffff   binit
00840b40   cinit
00800200   edata
00841044   end
0083df00   etext
ffffffff   pinit


GLOBAL SYMBOLS: SORTED BY Symbol Address 

address    name
--------   ----
00001000   __STACK_SIZE
00001000   __SYSMEM_SIZE
00800000   __CSL_intcVectorTable
00800200   .data
00800200   ___data__
00800200   ___edata__
00800200   _packet_header
00800200   edata
00801800   _packet_buffer
00831800   .text
00831800   ___text__
0083192c   _gblUserInit
008319c0   _main
00831ac8   _emac_Init
00832314   _emacTxPackets
00832594   _emacRxPackets
00832658   _closeEMAC
00832688   _EmacHwInt
008328f0   _EmacTimerTick
00832c40   _EMAC_open
00833600   _MDIO_timerTick
00834760   _CSL_intcHwControl
00834b20   _EMAC_close
00835220   __printfi
00835580   _MDIO_initPHY
00835ec0   _fputs
008361c0   _CSL_intcInit
00836d20   _free
00836fa0   _CSL_devHwControl
00837220   _EMAC_timerTick
00837480   _CSL_devGetHwStatus
008376e0   _CSL_tmrHwControl
00837940   _CSL_tmrHwSetup
00837ba0   _EMAC_serviceCheck
00837de0   __frcdivd
00838020   _CSL_intcOpen
00838260   _EmacTimerInitialization
00838340   _EmacInterruptsInitialization
00838448   _EmacInterruptEnd
00838480   __divull
00838d00   __CSL_intcEvent0Dispatcher
00838f20   __CSL_intcEvent1Dispatcher
00839140   __CSL_intcEvent2Dispatcher
00839360   __CSL_intcEvent3Dispatcher
00839580   __frcaddd
00839960   __CSL_intcDispatcher
00839b40   _EMAC_sendPacket
00839d00   __divd
00839ec0   _HOSTrename
0083a060   __divul
0083a200   __mpyd
0083a540   _setvbuf
0083a860   _malloc
0083a9e0   __addd
0083af60   __CSL_intcIvpSet
0083af70   _CSL_intcInterruptEnable
0083af90   _CSL_intcInterruptDisable
0083afb0   _CSL_intcInterruptClear
0083afc0   _CSL_intcInterruptSet
0083afcc   _CSL_intcInterruptRestore
0083afe4   _CSL_intcQueryInterruptStatus
0083aff8   _CSL_intcGlobalEnable
0083b018   _CSL_intcGlobalDisable
0083b038   _CSL_intcGlobalRestore
0083b050   _CSL_intcGlobalNmiEnable
0083b064   _CSL_intcGlobalExcepEnable
0083b078   _CSL_intcGlobalExtExcepEnable
0083b08c   _CSL_intcGlobalExcepClear
0083b0a0   _CSL_tmrGetHwSetup
0083b1e0   _EMAC_getStatus
0083b300   _EMAC_setReceiveFilter
0083b540   _fclose
0083b660   _fputc
0083b660   _putc
0083b780   _HOSTopen
0083b880   __frcmpyd
0083ba80   _atoi
0083bb80   _exit
0083bd80   _HOSTlseek
0083be60   __auto_init
0083c020   __wrt_ok
0083c100   _close
0083c2c0   _fseek
0083c3a0   _memset
0083c480   _HOSTread
0083c540   _HOSTunlink
0083c600   _HOSTwrite
0083c6c0   _MDIO_close
0083c780   __cleanup
0083c840   __divu
0083c9c0   _lseek
0083ca80   _ltoa
0083cb40   _write
0083cc00   _CSL_intcClose
0083ccc0   _CSL_tmrOpen
0083cd80   _HOSTclose
0083ce20   __divli
0083cec0   __doflush
0083d000   __fixdli
0083d0a0   __fltlid
0083d1e0   _memcpy
0083d3c0   _renormd
0083d460   _writemsg
0083d4e4   C$$IO$$
0083d500   _CSL_devOpen
0083d5a0   _MDIO_open
0083d620   __cmpd
0083d6a0   __fixdi
0083d720   __llshl
0083d7a0   _printf
0083d820   _readmsg
0083d8a0   _unlink
0083d920   __subcull
0083d980   _c_int00
0083d9e0   _memccpy
0083da40   _CSL_tmrGetBaseAddress
0083daa0   __args_main
0083dae0   __llshru
0083db20   __negd
0083db60   __remli
0083dba0   __strasgi_64plus
0083dbe0   __subd
0083dc60   _puts
0083dca0   _CACHE_setL1dSize
0083dce0   _CACHE_setL1pSize
0083dd20   _CACHE_setL2Size
0083dd60   _CSL_devGetBaseAddress
0083dda0   _MDIO_getStatus
0083ddc0   __negll
0083dde0   __nop
0083de40   C$$EXIT
0083de40   _abort
0083de60   _remove
0083de80   _CSL_devInit
0083dea0   __CSL_intcNmiDummy
0083dec0   _CSL_intcHookIsr
0083dee0   _CSL_tscEnable
0083dee8   _CSL_tscRead
0083df00   ___etext__
0083df00   __stack
0083df00   etext
0083ef00   __sys_memory
008401e0   __ftable
008402d0   __tmpnams
00840370   __ft_end
008406b8   __cleanup_ptr
008406bc   __dtors_ptr
008406c0   _LocalMAC
008406c8   _DestMAC
008406d0   _FreeQueue
008406dc   _RxQueue
0084074c   __lock
00840750   __unlock
00840a18   __ctypes_
00840b40   ___cinit__
00840b40   cinit
00840db8   __CIOBUF_
00840fb8   $bss
00840fb8   .bss
00840fb8   __CSL_intcAllocMask
00840fb8   ___bss__
00840fbc   __CSL_intcCpuIntrTable
00841000   __CSL_intcEventOffsetMap
00841004   __CSL_intcNumEvents
00841008   __CSL_intcEventHandlerRecord
0084100c   _uiTotalPacketsToTransfer
00841010   _uiTotalPacketsReceived
00841014   _EmacRegs
00841018   _EmacControlRegs
0084101c   _devRegs
00841020   _hEMAC
00841024   _LinkStatus
00841028   _LocalTicks
0084102c   _uiMacMode
0084103c   __CSL_cachebusyState
00841040   __CSL_cacheEmifState
00841044   ___end__
00841044   end
ffffffff   ___binit__
ffffffff   ___c_args__
ffffffff   ___pinit__
ffffffff   binit
ffffffff   pinit

[183 symbols]
